:100000000C9463000C948B000C948B000C948B006C
:100010000C948B000C948B000C948B000C94910727
:100020000C948B000C948B000C948B000C948B0024
:100030000C948B000C948B000C948B000C948B0014
:100040000C9447070C948B000C9415070C94EF0646
:100050000C948B000C948B000C948B000C948B00F4
:100060000C948B000C948B000000000023002600F1
:10007000290000000000240027002A0000000000E2
:10008000250028002B0004040404040404040202D4
:100090000202020203030303030301020408102007
:1000A0004080010204081020010204081020000012
:1000B0000008000201000003040700000000000027
:1000C000000051085E1711241FBECFEFD8E0DEBF3D
:1000D000CDBF23E0A0E7B1E001C01D92A639B20771
:1000E000E1F711E0A0E0B1E0E4E5FEE302C0059035
:1000F0000D92A037B107D9F710E0C2E6D0E004C0F6
:100100002197FE010E94381AC136D107C9F70E9413
:1001100091090C941D1F0C9400000895AF92BF929A
:10012000CF92DF92EF92FF920F931F93CF93DF93C3
:100130006C017B018B01040F151FEB015E01AE18F2
:10014000BF08C017D10759F06991D601ED91FC9114
:100150000190F081E02DC6010995892B79F7C50141
:10016000DF91CF911F910F91FF90EF90DF90CF9093
:10017000BF90AF900895FC01538D448D252F30E042
:10018000842F90E0821B930B541710F0CF960895A4
:1001900001970895FC01918D828D981761F0A28DD1
:1001A000AE0FBF2FB11D5D968C91928D9F5F9F7397
:1001B000928F90E008958FEF9FEF0895FC01918D4D
:1001C000828D981731F0828DE80FF11D858D90E0BA
:1001D00008958FEF9FEF0895FC01918D228D892F57
:1001E00090E0805C9F4F821B91098F73992708953F
:1001F0008EEB91E00E94EC0021E0892B09F420E0D5
:10020000822F0895FC01A48DA80FB92FB11DA35A08
:10021000BF4F2C91848D90E001968F739927848F26
:10022000A689B7892C93A089B1898C918370806449
:100230008C93938D848D981306C00288F389E02DEA
:1002400080818F7D80830895EF92FF920F931F939B
:10025000CF93DF93EC0181E0888F9B8D8C8D981379
:100260001AC0E889F989808185FF15C09FB7F89485
:10027000EE89FF896083E889F989808183708064D1
:1002800080839FBF81E090E0DF91CF911F910F911C
:10029000FF90EF900895F62E0B8D10E00F5F1F4F2B
:1002A0000F731127E02E8C8D8E110CC00FB607FC3A
:1002B000FACFE889F989808185FFF5CFCE010E94C8
:1002C0000201F1CFEB8DEC0FFD2FF11DE35AFF4F33
:1002D000F0829FB7F8940B8FEA89FB898081806256
:1002E000CFCFCF93DF93EC01888D8823B9F0AA8913
:1002F000BB89E889F9898C9185FD03C0808186FDE1
:100300000DC00FB607FCF7CF8C9185FFF2CF80812F
:1003100085FFEDCFCE010E940201E9CFDF91CF91A1
:100320000895833081F028F4813099F08230A9F06B
:1003300008958730A9F08830C9F08430B1F48091F5
:1003400080008F7D03C0809180008F778093800034
:10035000089584B58F7784BD089584B58F7DFBCFD4
:100360008091B0008F778093B00008958091B000A5
:100370008F7DF9CF1F93CF93DF93282F30E0F901C2
:10038000E255FF4F8491F901E656FF4FD491F901F0
:10039000EA57FF4FC491CC23A9F0162F81110E9478
:1003A0009101EC2FF0E0EE0FFF1FE458FF4FA591F5
:1003B000B4918FB7F894EC91111108C0D095DE2359
:1003C000DC938FBFDF91CF911F910895DE2BF8CF83
:1003D000CF93DF9390E0FC01E656FF4F24918A57BC
:1003E0009F4FFC0184918823D1F090E0880F991FE2
:1003F000FC01EE58FF4FA591B491FC01E458FF4F6A
:10040000C591D49161110EC09FB7F8948C91E22FE1
:10041000E0958E238C932881E223E8839FBFDF91B0
:10042000CF9108958FB7F894EC91E22BEC938FBFA6
:10043000F6CFCF93DF93EC0161E085E00E94E80105
:10044000209731F460E085E0DF91CF910C94BA0100
:10045000CF3FD10511F461E0F6CFE3EBF0E0E4919A
:10046000E33029F140F4E130B1F0E230D9F0C038A6
:10047000D1058CF7E7CFE73021F1E83051F1E430D6
:10048000B1F780918000806280938000D0938B00D0
:10049000C0938A0004C084B5806884BDC7BDDF9165
:1004A000CF91089584B5806284BDC8BDF8CF809196
:1004B0008000806880938000D0938900C09388007A
:1004C000EECF8091B00080688093B000C093B300FD
:1004D000E6CF8091B00080628093B000C093B400FA
:1004E000DECF8E3008F08E508770806480937C0061
:1004F00080917A00806480937A0080917A0086FDF2
:10050000FCCF809178009091790008953FB7F894DE
:100510008091750190917601A0917701B091780159
:1005200026B5A89B05C02F3F19F00196A11DB11D4E
:100530003FBFBA2FA92F982F8827BC01CD01620F8A
:10054000711D811D911D42E0660F771F881F991F45
:100550004A95D1F708958F929F92AF92BF92CF9212
:10056000DF92EF92FF926B017C010E9486024B01A9
:100570005C01C114D104E104F104B9F00E948602C7
:10058000681979098A099B09683E734081059105BC
:1005900080F321E0C21AD108E108F10888EE880E44
:1005A00083E0981EA11CB11CE4CFFF90EF90DF9078
:1005B000CF90BF90AF909F908F9008952FB7F894F1
:1005C0006091710170917201809173019091740139
:1005D0002FBF08958F929F92AF92BF92CF92DF92DA
:1005E000EF92FF920F931F936B017C010E94DE023A
:1005F00000915E0310915F032091600330916103CD
:100600004B015C01801A910AA20AB30A870130E00B
:1006100020E080169106A206B306F0F160935E0317
:1006200070935F038093600390936103609158031C
:100630007091590380915A0390915B039B01281B91
:10064000390BA90137FF04C044275527421B530B20
:10065000EC2DF0E08091520390915303813091058D
:1006600019F08430910521F581E0121613060CF47F
:1006700080E04E175F0714F0882331F180915D030D
:100680008F5F80935D0370935B0360935A0381E0F7
:1006900090915D039D1508F480E01F910F91FF90EC
:1006A000EF90DF90CF90BF90AF909F908F90089584
:1006B0000297029730F4832F8095881F8827881F20
:1006C000D8CF4E175F07D4F210925D03DCCFCF93E3
:1006D000DF93EC0188810E9471029A8389832B81C8
:1006E0003C81AC01421B530B9A0157FF03C031956B
:1006F000219531092230310514F09C838B838B8145
:100700009C81B0E0A0E02B853C85821B930BA10966
:10071000B109B7FF03C09C5FAF4FBF4F9A8789876E
:10072000BC0190E080E00E94C91720E030E044EB7B
:1007300053E40E942A1820E030E040E85AE30E9487
:100740002A186D837E838F839887DF91CF910895D8
:10075000CF93DF93CCE4D3E0198A8A819B810E94F6
:100760006703EA81FB81818592859F878E870E943E
:10077000DE026A8B7B8B8C8B9D8BDF91CF910895F2
:100780002091500330915103232BA1F522E030E05A
:100790003093530320935203909355038093540353
:1007A0000E94A8030E94DE026093620370936303B9
:1007B0008093640390936503E0914C03F0914D03A3
:1007C00085E998E0A0E0B0E085839683A783B087B1
:1007D00080E69AEEA0E0B0E0818B928BA38BB48B85
:1007E0008FEF9FEF968B858B81E090E09093510384
:1007F000809350030895CF93DF932091500330915D
:100800005103232B81F5C1E0D0E0D0935303C09373
:10081000520390935503809354030E94A8030E94AF
:10082000DE0260936203709363038093640390938A
:100830006503E0914C03F0914D0385E998E0A0E059
:10084000B0E085839683A783B08780E69AEEA0E028
:10085000B0E0818B928BA38BB48BD68BC58BD0935E
:100860005103C0935003DF91CF910895CF92DF924F
:10087000EF92FF920F931F93CF93DF93442331F1B5
:100880008C01D0E0C0E06B01770FEE08FF0861E05B
:1008900081E10E94BA01C701B6010E94AB0260E08B
:1008A00081E10E94BA0162E370E080E090E00E9482
:1008B000AB0221960C171D0751F7DF91CF911F91C5
:1008C0000F91FF90EF90DF90CF9008956E5C7F4F77
:1008D000072E000C880B990BDF91CF911F910F9180
:1008E000FF90EF90DF90CF900C94AB02EF92FF92CD
:1008F0000F931F93CF93DF937C0100EA11E0D0E0C8
:10090000C0E0F80161918F01C7018C0F9D1F0E940B
:10091000F0182196CE31D105A1F78EE190E0DF915C
:10092000CF911F910F91FF90EF90089580917E01DC
:1009300090917F010C9476040F931F93CF93DF93D4
:10094000C0EAD1E08C01005A1140C8018C0F9D1FF4
:100950000E94E818899381E0CE3BD807B1F78EE179
:1009600090E0DF91CF911F910F910895FC0180815C
:100970009181009711F00C94881760E070E0CB0132
:1009800008950F931F93CF93DF938C01EB01FC012C
:10099000808191810097E1F068817981611571050D
:1009A000A9F0428153812C813D814217530770F099
:1009B0000E94451C8C819D81F801958384831D8252
:1009C0001C82DF91CF911F910F9108950E94F61A1A
:1009D00088819981F801918380838A819B819383A7
:1009E00082838C819D8195838483198218821B82E6
:1009F0001A82E5CFCF93DF93EC018881998100972C
:100A000011F00E94F61A198218821D821C821B8224
:100A10001A82DF91CF910895FC0180819181009726
:100A200011F00C94F61A08950F931F93CF93DF9350
:100A3000EC0188819981009759F02A813B81261722
:100A4000370730F081E0DF91CF911F910F9108952A
:100A50008B016F5F7F4F0E947F1B009759F0998336
:100A600088831B830A832C813D81232B59F7FC014A
:100A70001082E8CF80E0E7CFEF92FF920F931F93B1
:100A8000CF93DF93EC01FB01E080F180E114F104EE
:100A900011F10481158101151105A9F08C819D8149
:100AA000080F191FB801CE010E941405882399F080
:100AB000288139818C819D81B701820F931F0E940B
:100AC000451C1D830C83CE01DF91CF911F910F91A7
:100AD000FF90EF900895CE010E94FA04F4CFEF92B8
:100AE000FF920F931F93CF93DF93EC017B018A0159
:100AF000BA010E94140581110BC0CE010E94FA04B4
:100B0000CE01DF91CF911F910F91FF90EF9008954B
:100B10001D830C83B701888199810E94451CF0CF09
:100B2000FC0111821082138212821582148250E01D
:100B300040E06EE671E00C946F05FB01019000202F
:100B4000E9F73197AF01461B570B0C946F05CF9314
:100B5000DF9300D0CDB7DEB7FC0111821082138283
:100B600012821582148269831A82BE016F5F7F4FE1
:100B70000E949D050F900F90DF91CF910895CF9324
:100B8000DF93EC01FB018617970749F060817181C3
:100B90006115710541F0448155810E946F05CE01B8
:100BA000DF91CF9108950E94FA04F9CFFF920F933D
:100BB0001F93CF93DF9300D0CDB7DEB786E0F82E3A
:100BC0008EEB91E00E94EC00892B09F476C08EEB4D
:100BD00091E00E94CA00833251F08E3309F049C07F
:100BE0006EE671E083E393E00E949D05E9CF2091DA
:100BF0002D0330912E0380913103909132032817F9
:100C00003907F4F640912F035091300320912B03C4
:100C100030912C03C901019690932C0380932B03F0
:100C2000F29EC001F39E900D112463E373E0840FE4
:100C3000951F0E94BF0580912D0390912E03019670
:100C400090932E0380932D0380912B0390912C037E
:100C50002091310330913203281739070CF0B0CFBF
:100C60002F5F3F4F821B930B90932C0380932B039A
:100C7000A7CF89831A8200913703109138030F5F41
:100C80001F4FB80183E393E00E941405882309F401
:100C900097CF2091330330913403809137039091A3
:100CA0003803BE016F5F7F4F820F931F0E94451C68
:100CB000109338030093370383CF0F900F90DF9189
:100CC000CF911F910F91FF9008950E94F80081111C
:100CD0000C94D60508950F931F93CF93DF93CDB750
:100CE000DEB7A0970FB6F894DEBF0FBECDBF1F9240
:100CF00093E29F937F936F93282F082E000C330B62
:100D00003F938F9389E491E09F938F931F9280E2AA
:100D10008F938E010F5F1F4F1F930F930E944C1CE8
:100D2000F80101900020E9F73197AF01401B510B0A
:100D3000B8018EEB91E00E948E000FB6F894DEBFF2
:100D40000FBECDBFA0960FB6F894DEBF0FBECDBFCD
:100D5000DF91CF911F910F9108950F931F93CF9320
:100D6000DF93CDB7DEB7A0970FB6F894DEBF0FBE06
:100D7000CDBF1F9293E29F937F936F93282F082EEE
:100D8000000C330B3F938F9381E591E09F938F93FA
:100D90001F9280E28F938E010F5F1F4F1F930F935F
:100DA0000E944C1CF80101900020E9F73197AF0137
:100DB000401B510BB8018EEB91E00E948E000FB6E4
:100DC000F894DEBF0FBECDBFA0960FB6F894DEBF7D
:100DD0000FBECDBFDF91CF911F910F9108951F924C
:100DE0000F920FB60F9211242F933F934F935F935F
:100DF0006F937F938F939F93AF93BF93EF93FF93E3
:100E00008EEB91E00E940201FF91EF91BF91AF91B3
:100E10009F918F917F916F915F914F913F912F9112
:100E20000F900FBE0F901F9018951F920F920FB644
:100E30000F9211242F938F939F93EF93FF93E09141
:100E4000CE01F091CF018081E091D401F091D501E4
:100E500082FD1BC090818091D7018F5F8F7320919D
:100E6000D801821741F0E091D701F0E0E254FE4F43
:100E7000958F8093D701FF91EF919F918F912F9143
:100E80000F900FBE0F901F9018958081F4CF1F9286
:100E90000F920FB60F9211242F933F938F939F932E
:100EA000AF93BF938091710190917201A0917301F2
:100EB000B09174013091700123E0230F2D3758F564
:100EC0000196A11DB11D2093700180937101909333
:100ED0007201A0937301B093740180917501909198
:100EE0007601A0917701B09178010196A11DB11D05
:100EF0008093750190937601A0937701B093780168
:100F0000BF91AF919F918F913F912F910F900FBE05
:100F10000F901F90189526E8230F0296A11DB11D72
:100F2000D2CF1F920F920FB60F9211242F933F939F
:100F30004F935F936F937F938F939F93AF93BF93E1
:100F4000CF93DF93EF93FF9320915B0230E0F901A1
:100F5000E255FF4F8491F901E656FF4FD491F90114
:100F6000EA57FF4FC491CC2379F081110E9491017F
:100F7000EC2FF0E0EE0FFF1FE859FF4FA591B49161
:100F8000EC91ED2381E009F480E020915E02309144
:100F90005F022F5F3F4F30935F0220935E0290917C
:100FA0002803943618F095E090935C0290915C02CF
:100FB000933009F44CC0E0F4923011F190915D024D
:100FC000992319F081116BC02D9AFF91EF91DF9158
:100FD000CF91BF91AF919F918F917F916F915F91D1
:100FE0004F913F912F910F900FBE0F901F9018952A
:100FF000943009F448C0953009F78111DFCF09C05A
:101000008111DCCF20915E0230915F0224363105E0
:1010100028F410925F0210925E02D0CF1092280343
:10102000E091280391E09E0F90932803F0E0209137
:101030005E0230915F02EE0FFF1FE55AFD4F3683CF
:10104000258310925F0210925E0293E019C08130F6
:1010500009F0B4CFE091280391E09E0F909328030C
:10106000F0E020915E0230915F02EE0FFF1FE55A23
:10107000FD4F3683258310925F0210925E0294E04A
:1010800090935C029BCF882359F220915E023091AD
:101090005F022536310508F491CF95E0F1CF2D9808
:1010A00094CFEF92FF920F931F93CF93DF93109201
:1010B000C1011092C00188EE93E0A0E0B0E08093FF
:1010C000C2019093C301A093C401B093C5012BE367
:1010D00031E03093BF012093BE0125EC30E0309326
:1010E000CB012093CA0124EC30E03093CD01209352
:1010F000CC0120EC30E03093CF012093CE0121ECE5
:1011000030E03093D1012093D00122EC30E03093D5
:10111000D3012093D20126EC30E03093D501209307
:10112000D4011092D7011092D8011092D9011092D7
:10113000DA0110927F0310928003109281031092C3
:1011400082031092830310928403109285031092FD
:1011500086031092870310928803109289031092DD
:101160008A0310928B0310928C0310928D031092BD
:101170008E0310928F0321E030E03093910320938F
:10118000900326E020937B0327E020937C0328E054
:1011900020937D0329E020937E032FE020936E03AC
:1011A0002EED33E030937A0320937903109270038D
:1011B00010926F03109272031092710310927803D1
:1011C00010927703109273031092740310927503B8
:1011D000109276032BE733E030934D0320934C03BA
:1011E0002EE633E030934F0320934E0310925103C9
:1011F0001092500310925703109256031092590305
:101200001092580310925B0310925A0310925C03E1
:1012100010925D0310925E0310925F0310926003C0
:1012200010926103109262031092630310926403A0
:101230001092650310926603109267031092680380
:101240001092690310926B0310926A0310926D035F
:1012500010926C0324E020935B0210925D022AE05E
:101260002093390310923A0380933B0390933C03FD
:10127000A0933D03B0933E0310923F0310924003AE
:1012800010924103109242031092430310924403C0
:10129000109245031092460384E690E0A0E0B0E08F
:1012A0008093470390934803A0934903B0934A0364
:1012B00010924B0383E393E00E94900510922A035F
:1012C0001092290310922C0310922B0310922E03DC
:1012D00010922D0384E190E09093320380933103C8
:1012E00080E890E00E945A1AEC0125E130E0299351
:1012F00039938E017C0120E8E20EF11CC8010E94A6
:1013000090050A5F1F4FE016F106C1F7D093300336
:10131000C0932F03DF91CF911F910F91FF90EF901A
:101320000895CF93DF93CDB7DEB7CD55D1090FB672
:10133000F894DEBF0FBECDBF789484B5826084BDC3
:1013400084B5816084BD85B5826085BD85B58160C9
:1013500085BD80916E00816080936E001092810047
:101360008091810082608093810080918100816002
:1013700080938100809180008160809380008091C3
:10138000B10084608093B1008091B000816080934F
:10139000B00080917A00846080937A0080917A0016
:1013A000826080937A0080917A00816080937A00D5
:1013B00080917A00806880937A001092C100E09159
:1013C000CE01F091CF0182E08083E091CA01F091DB
:1013D000CB011082E091CC01F091CD018FEC8083A4
:1013E0001092D601E091D201F091D30186E0808382
:1013F000E091D001F091D101808180618083E09102
:10140000D001F091D101808188608083E091D0018A
:10141000F091D101808180688083E091D001F091CA
:10142000D10180818F7D80838EEB91E00E94EC0062
:10143000892B29F08EEB91E00E94CA00F5CF61E084
:1014400081E10E94E80161E085E00E94E80161E03D
:1014500082E00E94E80161E08AE00E94E801AFE7D3
:10146000EA2EA3E0FA2E0BE713E061E0D8018D919C
:101470008D010E94E801F801319760E080810E94AF
:10148000BA01E016F10689F7EBE7F3E06496FFAFE7
:10149000EEAF649760E06496AEADBFAD64978D919A
:1014A0006496BFAFAEAF64970E94BA016496EEAD8A
:1014B000FFAD6497E017F10769F760E080916E0374
:1014C0000E94E80180916E030E9471029093700364
:1014D00080936F039093720380937103B0E0A0E058
:1014E0002091790330917A03821B930BA109B109F2
:1014F000B7FF03C09C5FAF4FBF4F909378038093BB
:101500007703BC0190E080E00E94C91720E030E042
:1015100044EB53E40E942A1820E030E040E85AE30C
:101520000E942A1860937303709374038093750369
:101530009093760380914E0390914F030E9467032E
:10154000E0914E03F0914F038185928590935B0368
:1015500080935A0361E0809139030E94E80160E0C2
:10156000809139030E94BA0188EE93E0A0E0B0E0D8
:1015700080933B0390933C03A0933D03B0933E03C1
:101580000E94DE02609343037093440380934503FB
:101590009093460381E080934B0384E690E0A0E0C3
:1015A000B0E08093470390934803A0934903B0931E
:1015B0004A036EE671E083E393E00E949D0510927A
:1015C0007F0110927E0110927D018EE190E0909358
:1015D0007C0180937B0182E290E090937A0180937A
:1015E000790110E000E0FF24F394C8010E949C04FC
:1015F0008091A0019091A1018336910531F410935F
:101600007F0100937E01F0927D01025E1F4F0C3F2F
:10161000F3E01F0751F700917E0110917F01809147
:101620007D01882309F46AC1C8010E949C041092BC
:10163000A1011092A001C8010E94760420917B01B3
:1016400030917C0180917E0190917F01820F931FE8
:1016500090937F0180937E016091790170917A016E
:10166000269FA001279F500D369F500D11248417EF
:10167000950724F010927F0110927E0183E690E09E
:101680009093A1018093A00180917E0190917F01B0
:101690000E9476048091AA01882321F061E082E013
:1016A0000E94BA0164E670E080E090E00E94AB0224
:1016B0008091A6019091A701019709F071C18091D5
:1016C000A8019091A9010E941902A091BC01A53620
:1016D00008F0A4E6A0933A0320913B0330913C0329
:1016E00040913D0350913E03B0E00E94FE1824E675
:1016F00030E040E050E00E94161A20933F03309300
:1017000040034093410350934203211531054105A5
:101710005105A9F08091470390914803A091490396
:10172000B0914A03281739074A075B0740F48093B2
:101730003F0390934003A0934103B0934203F89476
:1017400082E08093B0008093B10094E69093B30060
:101750001092B20080937000789480935C02109293
:10176000280380915B0260E00E94E8014091B5018E
:1017700066E970E081E090E00E94360480911F01EC
:1017800090912001A0912101B09122016A968CAF25
:101790009DAFAEAFBFAF6A978091230190912401B6
:1017A000A0912501B09126016E968CAF9DAFAEAF92
:1017B000BFAF6E9780912D0390912E0318161906D6
:1017C0000CF057C1CE01845B9F4F0E949005CE0163
:1017D0008A5B9F4F0E94900580912D0390912E036C
:1017E000009709F43CC18E010F5F1F4F18161906B0
:1017F0000CF4D9C0CE018E960E949005BE01625DA8
:101800007F4FCE01845B9F4F0E94C104CE018E9614
:101810000E940C056296CEACDFAC6297AA24A3941A
:10182000B12CC114D10421F05601CC24C394D12C85
:10183000C8010E9490056296EEACFFAC6297CE1490
:10184000DF0408F5AE14BF0408F475012E96EEAD62
:10185000FFAD2E97EE0DFF1DB08010822E966EAD5F
:101860007FAD2E976C0D7D1DC8016115710509F4C2
:10187000E4C00E949D052E968EAD9FAD2E97E80E7A
:10188000F91ED701BC92B801CE018A5B9F4F0E941E
:10189000C104C8010E940C0562968EAD9FAD62978F
:1018A000892B09F4DCC02E96EEADFFAD2E97309754
:1018B00009F4D5C0E081E254E83108F0D0C00E2E22
:1018C000000CFF0BEA59F34F0C94381AC00E810E2E
:1018D000B00E4B101A108111200D2F0DFB0E781138
:1018E0009A0E72101411680E2F0D2F0DAC100C0FE4
:1018F000420F2F0D5A0E8B11520F071083E690E006
:101900009093A1018093A00181E290E09093A301C4
:101910008093A20181E090E09093A5018093A401BF
:101920001092A7011092A6011092A9011092A8018D
:101930008093AA0122E030E03093AC012093AB0108
:1019400022E130E03093AE012093AD0120E430E09D
:101950003093B0012093AF0120E830E03093B20122
:101960002093B1012EEF30E03093B4012093B30106
:101970008093B5011092B7011092B6018DE290E00C
:101980009093B9018093B8018CEB92E09093BB01E6
:101990008093BA011092BD011092BC01C80178CEAB
:1019A00090E080E090CE2091290330912A0346E018
:1019B000429FC001439F900D112460912F037091AD
:1019C0003003680F791F1A8219821C821B821E82C3
:1019D0001D82C8010E94BF058091290390912A03AE
:1019E000019690932A038093290320912D0330912F
:1019F0002E032150310930932E0320932D03209183
:101A00003103309132032817390744F42F5F3F4FD9
:101A1000821B930B90932A03809329031FA61EA673
:101A200019AA18AA1BAA1AAAB801CE018E960E945A
:101A3000C104C8010E940C05E1CE0E94FA041BCF2C
:101A40006CE071E0C8010E94451C64E670E080E033
:101A500090E00E94AB02B80188E40E946B06CE01C0
:101A60008A5B9F4F0E940C05CE01845B9F4F0E94B2
:101A70000C0580E692E09093980180939701809105
:101A80002803282E312C30929A01209299018091BE
:101A90005C02853009F0DCC08091620290916302A3
:101AA000885891098D35910508F0ADC480912803BF
:101AB000843009F07AC48091640290916502809725
:101AC000479708F072C48091660290916702099767
:101AD000099708F06AC410929601109295018FEF51
:101AE0009FEFDC018093910190939201A093930169
:101AF000B093940181E090E090938E0180938D01EA
:101B00000E94DE024B015C01809191019091920153
:101B1000A0919301B09194018F3FEFEF9E07AE0724
:101B2000BE0709F006C58091890190918A01A091B4
:101B30008B01B0918C018093910190939201A093BD
:101B40009301B093940181E080938801C090890152
:101B5000D0908A01E0908B01F0908C0180918301FC
:101B600081112DC0FDE3CF16F2ECDF06FAE9EF0696
:101B7000F6EAFF0649F027E6C21628E9D2062AE966
:101B8000E20626EAF206D9F48091A6019091A70117
:101B9000019711F00C9498168091B6019091B701BD
:101BA000892B11F00C941D174091B50164E670E08B
:101BB00081E090E00E94360481E08093830147E653
:101BC000C41648E9D4064AE9E40646EAF40609F4EC
:101BD000FEC50CF0C9C49DEFC91692E0D9069AE97A
:101BE000E90696EAF90609F4FCC4ADEDCA16A2E2CC
:101BF000DA06AAE9EA06A6EAFA0611F40C94B9167E
:101C00008091A6019091A7010197E9F48091B60116
:101C10009091B701892BB9F48091A8019091A90105
:101C20008F3F910511F0019771F464E670E080E058
:101C300090E00E94AB024091B50164E670E082E062
:101C400090E00E94360482E080935C0210922803A8
:101C500080914B03882309F44CC60E94DE02009158
:101C600043031091440320914503309146036B01D7
:101C70007C01C01AD10AE20AF30A00913B031091D9
:101C80003C0320913D0330913E03C016D106E2068D
:101C9000F30640F06093430370934403809345033D
:101CA000909346032091390330913A03311103C6D2
:101CB00060E01CC668E071E0C8010E94451C64E653
:101CC00070E080E090E00E94AB02B80186E5C5CEEE
:101CD0004091B50168EC70E081E090E00E9436042C
:101CE00081E090E09093B7018093B6011092A50136
:101CF0001092A4018091BA019091BB010E94FB0354
:101D0000AECE4091B50168EC70E081E090E00E94B9
:101D1000360482E090E09093B7018093B601109270
:101D2000A5011092A4018091B8019091B9010E947F
:101D3000C00395CE81E090E09093A7018093A60127
:101D40000E9496048091A8019091A9010E94190215
:101D50006091A8017091A9018CE40E94AD067FCE2C
:101D60001092A7011092A6010E94960490E080E0D4
:101D70000E9419026091A8017091A90184E4EDCF3D
:101D8000CE018A5B9F4F0E94B60497FD2EC06F3F25
:101D900071058105910509F05CF57093A9016093C7
:101DA000A8018091A6019091A701019719F4CB0198
:101DB0000E9419020E9496048091A9018F9380913C
:101DC000A8018F9389E591E09F938F931F930F93C1
:101DD0000E947C1CB80182E40E946B060F900F9059
:101DE0000F900F900F900F903ACE70E060E0D5CF3B
:101DF0006FEF70E0D2CF8091A9018F938091A801FD
:101E00008F9389E591E09F938F931F930F930E9487
:101E10007C1CB8018AE4E0CF8091BB018F93809154
:101E2000BA018F938091B9018F938091B8018F93FC
:101E30008091BD018F938091BC018F938091A5010A
:101E40008F938091A4018F938091A7018F938091AC
:101E5000A6018F938091B7018F938091B6018F93E4
:101E60008CE591E09F938F931F930F930E947C1CAE
:101E7000B80183E50E946B060FB6F894DEBF0FBE73
:101E8000CDBFEDCDCE018A5B9F4F0E94B604672B7C
:101E900029F41092B5010E949604E1CD81E080936F
:101EA000B501F9CF6BEAC62E61E0D62E72E0E72EBF
:101EB000F12C2C968EAD9FAD2C97E816F90638F4D0
:101EC0002896EEADFFAD2897309709F091C010929B
:101ED0008001E0E8F1E06081C8010E94A705C70128
:101EE00001972C962EAD3FAD2C978217930738F4AF
:101EF0002896EEADFFAD2897309709F07CC0109280
:101F00008001E0E8F1E06081CE018E960E94A70595
:101F1000C70102972C962EAD3FAD2C9782179307E1
:101F200038F42896EEADFFAD2897309709F066C0DB
:101F300010928001E0E8F1E06081CE01CA960E9433
:101F4000A7051DAA1CAA1FAA1EAA19AE18AEBE017B
:101F5000665C7F4FCE01C4960E94BF05BE01625DE4
:101F60007F4FCE01C4960E943C05B8010E943C05FB
:101F700022961FAE1EAE229724961FAE1EAE249749
:101F800026961FAE1EAE2697BC01CE01805C9F4FE9
:101F90000E94BF05CE01C4960E940C05CE01CA96D0
:101FA0000E940C05CE018E960E940C05C8010E946D
:101FB0000C05CE01805C9F4F0E94B60497FD21C0A6
:101FC0006F3F71058105910509F0F4F4D6016D9319
:101FD0007D936D01CE01805C9F4F0E940C05B3E0A4
:101FE000EB0EF11CE1E1EE16F10409F062CF53CFE4
:101FF000EE0DFF1D70CFE80FF91F85CFE80FF91F19
:102000009BCF70E060E0E2CF6FEF70E0DFCFCE01FA
:102010008A5B9F4F0E94B604672B39F41092AA0185
:1020200060E082E00E94BA0136CF81E08093AA018D
:1020300061E0F7CF8EE693E00E946703809177031B
:10204000909178039C01215031092F36334000F5DF
:102050009093B9018093B8011092B7011092B60124
:1020600081E090E09093A5018093A4010E949604E2
:102070006091B8017091B90186E40E94AD0640916B
:10208000B50164E670E082E090E00E943604E7CC9F
:102090008DE290E0DDCF8EE693E00E9467038091B1
:1020A0007703909178039C01215031092F363340FA
:1020B000B0F49093BB018093BA011092B7011092D3
:1020C000B60182E090E09093A5018093A4010E9464
:1020D00096046091BA017091BB0185E4CECF8CEB80
:1020E00092E0E7CFCE018A5B9F4F0E94B604072E95
:1020F000000C880B990B0E94CB172AE43CE046E3C6
:1021000050E40E942A1820E030E040E05FE30E94A3
:1021100050190E94BC196B018EE693E00E94670380
:102120001092A5011092A4018091770390917803F9
:10213000D7FE09C022E030E03093B7012093B6010A
:102140008C0D9D1DF4CD21E030E03093B70120933C
:10215000B6018C0D9D1DD2CD4091B50168EC70E0AB
:1021600081E090E00E9436048091500390915103E9
:10217000892B09F052C084E090E090935303809340
:1021800052030E94A8030E94DE02609362037093D0
:1021900063038093640390936503E0914C03F09193
:1021A0004D0385E998E0A0E0B0E085839683A7839E
:1021B000B08780914E0390914F030E946703E09196
:1021C0004E03F0914F03818592859093570380933E
:1021D000560310925C03E0914C03F0914D0385850A
:1021E0009685A785B0898093660390936703A09333
:1021F0006803B093690380E69AEEA0E0B0E0818BBB
:10220000928BA38BB48B81E090E0968B858B83E0DF
:1022100090E0909351038093500384E090E090937A
:10222000B7018093B6011BCC4091B50168EC70E01A
:1022300081E090E00E943604809150039091510318
:10224000892B09F052C083E090E090935303809370
:1022500052030E94A8030E94DE02609362037093FF
:1022600063038093640390936503E0914C03F091C2
:102270004D0385E998E0A0E0B0E085839683A783CD
:10228000B08780914E0390914F030E946703E091C5
:102290004E03F0914F03818592859093570380936D
:1022A000560310925C03E0914C03F0914D03858539
:1022B0009685A785B0898093660390936703A09362
:1022C0006803B093690380E69AEEA0E0B0E0818BEA
:1022D000928BA38BB48B8FEF9FEF968B858B82E0D5
:1022E00090E0909351038093500383E090E097CF68
:1022F00010928C0310928D0310928E0310928F0314
:10230000AECB8EE693E00E946703609177037091F5
:10231000780387E422CDCE018A5B9F4F0E94B604EA
:10232000DB0177FF02C0B0E0A0E0A536B10514F0F4
:10233000A4E6B0E0B093BD01A093BC01A0933A0322
:1023400020913B0330913C0340913D0350913E036B
:102350000E943E1A24E630E040E050E00E94161A47
:1023600020933F0330934003409341035093420333
:10237000211531054105510509F48DCD80914703A3
:1023800090914803A0914903B0914A032817390757
:102390004A075B0708F07FCD80933F03909340038B
:1023A000A0934103B093420376CD809128038434F7
:1023B00050F18091640290916502825491098E9748
:1023C00010F530E020E080E090E0DC01F901EA590E
:1023D000FD4F40815181495051094930510598F4D0
:1023E000F901E859FD4F4081518146515109413170
:1023F000510508F476C0408151814650510947305B
:10240000510508F480C096E0291631040CF41BCC69
:10241000ABE5B2E06696BFAFAEAF669703E010E003
:1024200035ECC32E3DE9D32E3CE1E32E31E8F32E0B
:10243000021513050CF06CC06696EEADFFAD669705
:1024400063857485A780B08490E080E00E94C917FE
:102450002B013C01B50190E080E00E94C9174B01BF
:102460005C012DEC3CEC4CE45FE30E942A189B01DC
:10247000AC01C301B2010E94C417F0E0E0E087FDA7
:1024800014C02DEC3CEC4CE45FE3C301B2010E94AC
:102490002A189B01AC01C501B4010E94C417E2E0F7
:1024A000F0E087FD02C0E1E0F0E0A701960163E9FA
:1024B00071E080E091E00E94F2196F01FF0FEE08D9
:1024C000FF08C626D726E826F9260F5F1F4F669617
:1024D0008EAD9FAD6697029666969FAF8EAF66975C
:1024E000A7CF880F991FAA1FBB1F81602C5F3F4F8A
:1024F0002038310509F06ACF20E230E030939601B0
:1025000020939501EFCA880F991FAA1FBB1FEECF1A
:10251000C0929101D0929201E0929301F0929401C5
:1025200080E290E090939601809395018FEF9FEF6A
:10253000E3CA8093890190938A01A0938B01B093A1
:102540008C011092880180E991E0909301018093C1
:1025500000018092840190928501A0928601B09240
:10256000870110928301F2CAB7E5CB16B8EADB0601
:10257000BAE9EB06B6EAFB0609F495C0EDE3CE1620
:10258000E2ECDE06EAE9EE06E6EAFE0609F41FC121
:10259000FDE5CF16F2EADF06FAE9EF06F6EAFF06F6
:1025A00009F02ECB4091B50164E670E081E090E047
:1025B0000E9436048091A4019091A501813091057B
:1025C00009F0EAC09093B7018093B6011092A5017B
:1025D0001092A4018091BA019091BB010E94FB036B
:1025E0000FCB8091B6019091B701892B09F008CBF0
:1025F0004091B50164E670E081E090E00E9436040D
:102600008091A6019091A701892B99F481E090E037
:102610009093A7018093A6018FEF9FEF9093820183
:10262000809381018091A8019091A9010E941902D3
:10263000AFC01092A7011092A60190E080E0F6CF03
:102640000E94DE02C0908401D0908501E090860156
:10265000F0908701AB01BC014C195D096E097F093F
:102660008091000190910101B0E0A0E04817590766
:102670006A077B0708F091C3C3CA8091AA01811140
:10268000BFCA11E01093AA0161E082E00E94BA0182
:102690004091B50164E670E082E090E00E9436046B
:1026A00010939F01ADCA8091A6019091A701019757
:1026B00009F0C9CA8091B6019091B701892B09F040
:1026C000A5CA10918801111133C00E94DE026093E7
:1026D0008401709385018093860190938701111185
:1026E00044C04091B50164E670E081E090E00E9452
:1026F000360400918101109182011016110614F028
:1027000001E010E001501109109382010093810152
:102710000115110509F468C3000F111FF801E056F7
:10272000FE4F838594859093A9018093A8017ECF65
:102730000E94DE02C0908401D0908501E090860165
:10274000F0908701AB01BC014C195D096E097F094E
:102750008091000190910101B0E0A0E04817590775
:102760006A077B0708F0B1CF4BCA8091AA01882382
:1027700009F446CA1092AA0160E082E00E94BA0100
:102780004091B50164E670E082E090E00E9436047A
:1027900081E080939F0134CA8230910579F490934F
:1027A000B7018093B6011092A5011092A401809107
:1027B000B8019091B9010E94C00322CA10928C0303
:1027C00010928D0310928E0310928F0319CA80917C
:1027D000A6019091A701019709F035CA8091B60131
:1027E0009091B701892B09F011CA1091880111232A
:1027F000D1F08091840190918501A0918601B091E2
:102800008701B501A401481B590B6A0B7B0B809112
:10281000000190910101B0E0A0E0481759076A0754
:102820007B0708F4F3C98092840190928501A092FD
:102830008601B09287013091A8012091A901832FD0
:10284000922F4DE3C41642ECD4064AE9E40646EA68
:10285000F40639F58F3F910514F08EEF90E0019664
:102860009093A9018093A8018091A8019091A9015A
:102870000E94190281E080939F01112309F4C0C9CD
:1028800080910001909101018333910508F4B8C94A
:1028900044978233910560F0909301018093000189
:1028A000AFC98230910514F482E090E00197D8CF4F
:1028B00082E390E0F1CFC0904303D0904403E090D6
:1028C0004503F09046036C197D098E099F09C0905D
:1028D0003F03D0904003E0904103F09042036C1519
:1028E0007D058E059F0508F0E3C961E0822F0E94F7
:1028F000BA018091500390915103892B11F10E94EC
:10290000DE02009162031091630320916403309111
:102910006503601B710B820B930B6135734C810552
:10292000910508F431C1E0914C03F0914D03118AF7
:10293000128A138A148A85E090E090935103809361
:10294000500380918C0390918D03A0918E03B091E0
:102950008F03892B8A2B8B2B09F48DC080918003E8
:1029600090918103A0918203B0918303892B8A2BDC
:102970008B2B09F480C00E94860200918403109181
:10298000850320918603309187036B017C01C01A77
:10299000D10AE20AF30A0091800310918103209189
:1029A000820330918303C016D106E206F30608F4D1
:1029B00062C0609384037093850380938603909331
:1029C000870380917F032091900330919103820FC0
:1029D000932F911D049664E070E00E94021A809388
:1029E0007F038C011127000F111F000F111F095DBC
:1029F0001E4F9BE7E92E93E0F92EF80161918F01BC
:102A0000D7018D917D010E94BA016496EEADFFADB4
:102A10006497EE16FF0689F78091900390919103D9
:102A2000092E000CAA0BBB0B40918803509189031F
:102A300060918A0370918B03840F951FA61FB71FA7
:102A40008093880390938903A0938A03B0938B03A8
:102A500080918C0390918D03A0918E03B0918F0390
:102A60000197A109B10980938C0390938D03A093E2
:102A70008E03B0938F03809150039091510304977C
:102A8000029708F045C08EE693E00E9467038091AC
:102A9000B6019091B7018230910509F421C108F087
:102AA000EFC0019709F40EC180915003909151033A
:102AB000059731F483E090E09093A5018093A40101
:102AC0001092B7011092B60100914C0310914D0382
:102AD000780184E0E80EF11C60E0D8018D918D0151
:102AE0000E94BA01E016F106B9F710925103109254
:102AF000500310925C0310925D0381E080939F016C
:102B00004091B50164E670E082E090E00E943604F6
:102B100080919F01813071F50E94DE0200919B013E
:102B200010919C0120919D0130919E016B017C01CF
:102B3000C01AD10AE20AF30AB9E8CB16B3E1DB0600
:102B4000E104F10428F4601771078207930790F4F9
:102B500060939B0170939C0180939D0190939E01D3
:102B600083E690E09093A1018093A0010E949604D7
:102B700010929F010E94F800882311F40C94DA0B44
:102B80000E94D6050C94DA0B80914E0390914F036E
:102B90000E946703E0914E03F0914F032185328537
:102BA000309359032093580380915003909151031F
:102BB0000197F1F480915403909155034091520391
:102BC000509153034130510509F04EC00296281729
:102BD0003907E0F1E0914C03F0914D03118A128A1C
:102BE000138A148A84E090E09093510380935003F9
:102BF00080915003909151030297029708F0A1CE63
:102C00006A966CAD7DAD8EAD9FAD6A970E94EA026B
:102C1000882309F496CEE0914C03F0914D03118A7C
:102C2000128A138A148A8091580390915903209133
:102C300050033091510323303105E1F40397909311
:102C40006B0380936A0384E090E077CE20373340B3
:102C500008F66E966CAD7DAD8EAD9FAD6E970E9401
:102C6000EA028111B7CFC4CF02978217930708F009
:102C7000B1CFEFCF039690936D0380936C03E3CFB6
:102C800083309105C9F1049709F00ECF82E090E0FE
:102C90009093A5018093A40180916A0390916B03A6
:102CA0009C01215031092F36334010F08CEB92E01B
:102CB0009093BB018093BA016091BA017091BB01FE
:102CC00082E50BC082E090E09093A5018093A4017F
:102CD00060917703709178038FE40E94AD06E4CE93
:102CE00081E090E09093A5018093A4016091770327
:102CF0007091780383E4F1CF81E090E09093A50197
:102D00008093A40180916C0390916D039C012150EC
:102D100031092F36334010F08DE290E09093B901E5
:102D20008093B8016091B8017091B9018EE4D5CF5C
:102D3000E7E6CE16E8E9DE06EAE9EE06E6EAFE0692
:102D400009F445CD0CF059C02DEFC21622E0D20691
:102D50002AE9E20626EAF20609F443CC4DEDC41650
:102D600042E2D4064AE9E40646EAF40611F00C947D
:102D7000230E8091A6019091A701019711F00C9468
:102D8000230E8091B6019091B701892B11F00C941C
:102D9000060E10918801111153CC0E94DE0260933F
:102DA00084017093850180938601909387011111AE
:102DB00064CC4091B50164E670E081E090E00E944F
:102DC000360400918101109182010430110514F044
:102DD00003E010E00F5F1F4F109382010093810109
:102DE0000430110509F098CC4091B50164E670E01B
:102DF00082E090E00E9436048FCC87E5C81688EA0E
:102E0000D8068AE9E80686EAF80609F44CCC9DE380
:102E1000C91692ECD9069AE9E90696EAF90609F488
:102E2000D6CCADE5CA16A2EADA06AAE9EA06A6EA0F
:102E3000FA0609F4B7CB0C94230EB7E6CB16B8E923
:102E4000DB06BAE9EB06B6EAFB0609F4C0CCB4F43B
:102E5000FDEFCF16F2E0DF06FAE9EF06F6EAFF062D
:102E600009F4BFCB2DEDC21622E2D2062AE9E20612
:102E700026EAF20609F47DCF0C94060E47E5C41647
:102E800048EAD4064AE9E40646EAF40609F40BCC1B
:102E90008DE3C81682ECD8068AE9E80686EAF806C9
:102EA00009F495CC9DE5C91692EAD9069AE9E90696
:102EB00096EAF90609F476CB0C94060ECF93DF93CD
:102EC000C0912F03D09130032097E1F0FE0132979B
:102ED0002081318146E0429FC001439F900D112423
:102EE000C80FD91F9E0180912F0390913003269720
:102EF0008217930721F0CE010E940C05F3CF0297B1
:102F00000E94F61A83E393E0DF91CF910C940C05B5
:102F10001F93FC0199278827BC01E8941191103276
:102F2000E9F3193010F01E30C8F31B3251F01D3296
:102F300049F4689406C00E94AF17610F711D811D8E
:102F4000911D119110531A30B0F33EF49095809575
:102F5000709561957F4F8F4F9F4F1F910895592F07
:102F6000482F372F262F660F771F881F991F660F50
:102F7000771F881F991F620F731F841F951F660F8D
:102F8000771F881F991F08950E94061808F481E092
:102F90000895E89409C097FB3EF49095809570954C
:102FA00061957F4F8F4F9F4F9923A9F0F92F96E995
:102FB000BB279395F695879577956795B795F1110A
:102FC000F8CFFAF4BB0F11F460FF1BC06F5F7F4FA7
:102FD0008F4F9F4F16C0882311F096E911C07723B9
:102FE00021F09EE8872F762F05C0662371F096E8C2
:102FF000862F70E060E02AF09A95660F771F881F91
:10300000DAF7880F9695879597F90895990F000834
:10301000550FAA0BE0E8FEEF16161706E807F907AA
:10302000C0F012161306E407F50798F0621B730B45
:10303000840B950B39F40A2661F0232B242B252BC6
:1030400021F408950A2609F4A140A6958FEF811D69
:10305000811D08950E943D180C94AE180E94A0187E
:1030600038F00E94A71820F0952311F00C949718BF
:103070000C949D1811240C94E2180E94BF1870F350
:10308000959FC1F3950F50E0551F629FF001729F0D
:10309000BB27F00DB11D639FAA27F00DB11DAA1F1C
:1030A000649F6627B00DA11D661F829F2227B00D69
:1030B000A11D621F739FB00DA11D621F839FA00DF4
:1030C000611D221F749F3327A00D611D231F849F44
:1030D000600D211D822F762F6A2F11249F5750409B
:1030E0009AF0F1F088234AF0EE0FFF1FBB1F661F16
:1030F000771F881F91505040A9F79E3F510580F0DF
:103100000C9497180C94E2185F3FE4F3983ED4F3C4
:10311000869577956795B795F795E7959F5FC1F782
:10312000FE2B880F911D9695879597F9089597F92D
:103130009F6780E870E060E008959FEF80EC08955D
:1031400000240A9416161706180609060895002486
:103150000A9412161306140605060895092E039400
:10316000000C11F4882352F0BB0F40F4BF2B11F474
:1031700060FF04C06F5F7F4F8F4F9F4F089557FDD3
:103180009058440F551F59F05F3F71F04795880FD5
:1031900097FB991F61F09F3F79F08795089512166C
:1031A00013061406551FF2CF4695F1DF08C0161618
:1031B00017061806991FF1CF8695710561050894C9
:1031C0000895E894BB2766277727CB0197F90895E0
:1031D000F999FECF92BD81BDF89A992780B50895DF
:1031E000262FF999FECF1FBA92BD81BD20BD0FB623
:1031F000F894FA9AF99A0FBE019608950E94401920
:10320000A59F900DB49F900DA49F800D911D11243A
:1032100008952F923F924F925F926F927F928F927A
:103220009F92AF92BF92CF92DF92EF92FF920F9355
:103230001F93CF93DF93CDB7DEB7CA1BDB0B0FB65F
:10324000F894DEBF0FBECDBF09942A88398848881C
:103250005F846E847D848C849B84AA84B984C884B2
:10326000DF80EE80FD800C811B81AA81B981CE0FA9
:10327000D11D0FB6F894DEBF0FBECDBFED0108958E
:10328000A29FB001B39FC001A39F700D811D1124A7
:10329000911DB29F700D811D1124911D08955058EC
:1032A000BB27AA270E9467190C94AE180E94A01889
:1032B00038F00E94A71820F039F49F3F19F426F443
:1032C0000C949D180EF4E095E7FB0C949718E92FE9
:1032D0000E94BF1858F3BA1762077307840795074F
:1032E00020F079F4A6F50C94E1180EF4E0950B2E7D
:1032F000BA2FA02D0B01B90190010C01CA01A00148
:103300001124FF27591B99F0593F50F4503E68F1A2
:103310001A16F040A22F232F342F4427585FF3CFE3
:10332000469537952795A795F0405395C9F77EF4B4
:103330001F16BA0B620B730B840BBAF09150A1F0FD
:10334000FF0FBB1F661F771F881FC2F70EC0BA0F83
:10335000621F731F841F48F4879577956795B7950B
:10336000F7959E3F08F0B0CF9395880F08F0992706
:10337000EE0F9795879508950E94C3196894B1112F
:103380000C94E21808950E94C71888F09F5798F08F
:10339000B92F9927B751B0F0E1F0660F771F881F5A
:1033A000991F1AF0BA95C9F714C0B13091F00E9474
:1033B000E118B1E008950C94E118672F782F882761
:1033C000B85F39F0B93FCCF3869577956795B3959B
:1033D000D9F73EF490958095709561957F4F8F4F0A
:1033E0009F4F0895DB018F939F930E94FE18BF911A
:1033F000AF91A29F800D911DA39F900DB29F900D44
:103400001124089597FB072E16F4009407D077FD3A
:1034100009D00E94461A07FC05D03EF4909581958C
:103420009F4F0895709561957F4F0895A1E21A2EE0
:10343000AA1BBB1BFD010DC0AA1FBB1FEE1FFF1F58
:10344000A217B307E407F50720F0A21BB30BE40BA8
:10345000F50B661F771F881F991F1A9469F76095EF
:103460007095809590959B01AC01BD01CF010895A9
:10347000EE0FFF1F0590F491E02D0994B7FF0C9417
:10348000FE180E94FE18821B930B0895AA1BBB1BFB
:1034900051E107C0AA1FBB1FA617B70710F0A61B54
:1034A000B70B881F991F5A95A9F780959095BC0175
:1034B000CD0108950F931F93CF93DF938230910531
:1034C00010F482E090E0E0919403F091950330E0F5
:1034D00020E0B0E0A0E0309799F42115310509F41F
:1034E0004AC0281B390B24303105D8F58A819B81CD
:1034F0006115710589F1FB0193838283FE0111C07F
:10350000408151810281138148175907E0F0481723
:10351000590799F4109761F012960C93129713962D
:103520001C933296CF01DF91CF911F910F91089597
:103530000093940310939503F4CF2115310551F0B6
:103540004217530738F0A901DB019A01BD01DF01E1
:10355000F801C1CFEF01F9CF9093950380939403C5
:10356000CDCFFE01E20FF31F8193919322503109D9
:1035700039832883D7CF2091920330919303232B53
:1035800041F420910401309105013093930320937D
:10359000920320910201309103012115310541F47C
:1035A0002DB73EB74091060150910701241B350B02
:1035B000E0919203F0919303E217F307A0F42E1B1E
:1035C0003F0B2817390778F0AC014E5F5F4F241787
:1035D000350748F04E0F5F1F5093930340939203BB
:1035E000819391939FCFF0E0E0E09CCFCF93DF9366
:1035F0000097E9F0FC01329713821282A0919403A4
:10360000B0919503ED0130E020E01097A1F4208106
:103610003181820F931F20919203309193032817D9
:10362000390709F061C0F0939303E0939203DF91AF
:10363000CF910895EA01CE17DF07E8F54A815B8153
:103640009E0141155105B1F7E901FB83EA834991D8
:103650005991C40FD51FEC17FD0761F4808191814A
:103660000296840F951FE901998388838281938153
:103670009B838A83F0E0E0E012968D919C911397F2
:103680000097B9F52D913C911197CD010296820FCB
:10369000931F20919203309193032817390739F62D
:1036A000309751F51092950310929403B0939303C1
:1036B000A0939203BCCFD383C28340815181840FF6
:1036C000951FC817D90761F44E5F5F4F88819981B4
:1036D000480F591F518340838A819B819383828342
:1036E0002115310509F0B0CFF0939503E0939403D1
:1036F0009ECFFD01DC01C0CF13821282D7CFB0E094
:10370000A0E0E5E8FBE10C940B198C01009751F463
:10371000CB010E945A1A8C01C801CDB7DEB7E0E197
:103720000C942719FC01E60FF71F9C012250310968
:10373000E217F30708F49DC0D901CD91DC911197F0
:10374000C617D70798F0C530D10530F3CE010497DE
:103750008617970708F3C61BD70B2297C193D193FF
:103760006D937C93CF010E94F61AD6CF5B01AC1A01
:10377000BD0A4C018C0E9D1EA0919403B09195033F
:10378000512C412CF12CE12C109731F580919203B2
:10379000909193038815990509F05CC04616570669
:1037A00008F058C08091020190910301009741F404
:1037B0008DB79EB74091060150910701841B950B70
:1037C000E817F90708F055C0F0939303E0939203CC
:1037D000F90171836083A0CF8D919C91119712960E
:1037E0006C90129713967C901397A815B90559F50C
:1037F0006C0142E0C40ED11CCA14DB0420F1AC0100
:103800004A195B09DA011296159780F06282738279
:1038100051834083D9016D937C93E114F10471F0DD
:10382000D7011396FC93EE93129776CF22968C0FC6
:103830009D1FF90191838083F301EFCFF0939503EE
:10384000E093940369CF4816590608F42C017D01D2
:10385000D3019ACFCB010E945A1A7C01009749F0FC
:10386000AE01B8010E943C1CC8010E94F61A8701F3
:1038700053CF10E000E050CFFB01DC0102C001900B
:103880000D9241505040D8F70895FB01DC010190A2
:103890000D920020E1F70895AEE0B0E0E2E5FCE132
:1038A0000C9417190D891E898F89988D26E02C8319
:1038B0001A83098397FF02C080E090E801979E83F6
:1038C0008D83AE01455E5F4F698D7A8DCE01019685
:1038D0000E949F1C4D815E8157FD0AC02F81388553
:1038E000421753070CF49A01020F131FF8011082BC
:1038F0002E96E4E00C943319AEE0B0E0E2E8FCE18F
:103900000C9417190D891E8986E08C831A8309830C
:103910008FEF9FE79E838D83AE01475E5F4F6F8978
:10392000788DCE0101960E949F1C2F813885020F51
:10393000131FF80110822E96E4E00C943319ABE0CB
:10394000B0E0E5EAFCE10C9409197C013B018A0135
:10395000FC0117821682838181FFC8C1CE010196C6
:103960005C01F7019381F30193FD859193FF8191B0
:103970003F01882309F453C1853239F493FD8591C1
:1039800093FF81913F01853229F4B70190E00E94B5
:103990008F1EE7CF912C212C312CFFE1F31538F04D
:1039A0008B3211F190F4803209F1833229F137FC26
:1039B0003CC020ED280F2A3050F536FE20C08AE0AA
:1039C000989E200D1124922E06C08D3291F08033E6
:1039D00071F7689430F8F30193FD859193FF81911D
:1039E0003F018111DACF21C0689431F8689432F830
:1039F000F2CF689433F8EFCF689434F8ECCFEAE074
:103A00002E9E200D1124222E689435F8E4CF8E329C
:103A100029F436FC04C1689436F8DDCF8C3619F4ED
:103A2000689437F8D8CF8836B1F2982F9F7D955497
:103A30009330E0F08336A1F18337C1F1833509F08B
:103A400063C02801F2E04F0E511CF801C080D18004
:103A5000692D70E036FC02C06FEF7FEFC6010E9457
:103A6000791E4C01689437F882010AC00C5F1F4F21
:103A7000FFE3F98388248394912C6501E89437F857
:103A800033FE2DC0522C8114910471F5552009F498
:103A900068CFB70180E290E00E948F1E5A94F6CF63
:103AA000F801808189830E5F1F4FE4CF2801F2E087
:103AB0004F0E511CF801C080D180692D70E036FC9A
:103AC00002C06FEF7FEFC6010E94841E4C0182018D
:103AD000D5CFB70180E290E00E948F1E2A9428146F
:103AE000190409F0B0F7CECFF60137FC859137FE07
:103AF00081916F01B70190E00E948F1E51105A947E
:103B0000F1E08F1A9108BFCF843619F0893609F099
:103B100077C0F80137FE6BC060817181828193812B
:103B20000C5F1F4FF32DFF763F2E97FF09C0909536
:103B30008095709561957F4F8F4F9F4F689437F8B0
:103B40002AE030E0A5010E94BF1EC82ECA188C2CA6
:103B5000432C36FE0CC0E89440F8C91440F434FEFF
:103B600005C032FC03C0F32DFE7E4F2E892C44FE8F
:103B700095C0FE01EC0DF11D8081803309F087C0F6
:103B8000242D297E422E842D8870582E43FC95C00A
:103B900040FE8FC09C2C821418F42C0C922C981888
:103BA00044FE91C0B70180E390E00E948F1E42FE68
:103BB00009C088E790E041FE02C088E590E0B701C7
:103BC0000E948F1EC91408F48AC0CA94D12C9FEF9A
:103BD000C91AD90ACA0CDB1CF60182916F01B70120
:103BE00090E00E948F1EAC14BD04B1F74FCF6081EE
:103BF0007181072E000C880B990B0E5F1F4F92CF1F
:103C0000D32CE894D4F82AE030E0853739F1232D1D
:103C1000297FD22E8F3601F148F48835A9F0F701BB
:103C2000868197812B96E2E10C942519803749F023
:103C30008837A9F7D4FE02C06894D2F820E130E0BA
:103C40000DC06894D4F8F6CF34FE03C0822F86608E
:103C5000D82E20E132E002C028E030E0F801D7FEA3
:103C60000FC060817181828193810C5F1F4FA5011C
:103C70000E94BF1EC82ECA183D2CE89437F867CFA3
:103C80006081718190E080E00E5F1F4FF0CF42FCB9
:103C900002C0839478CF8394839475CF842D8678E3
:103CA00009F471CFF6CFB70180E290E00E948F1E39
:103CB00083948214C0F3512C73CF522C5818821461
:103CC00008F46ECFF8CF842D867809F47BCF8BE291
:103CD00041FE80E247FC8DE2B70190E071CFB70171
:103CE00080E390E00E948F1E9A946CCF8FEF9FEF3D
:103CF00099CFFC010590615070400110D8F7809574
:103D000090958E0F9F1F0895FC01615070400190A7
:103D10000110D8F7809590958E0F9F1F08950F93EF
:103D20001F93CF93DF93182F092FEB018B8181FD18
:103D300009C01FEF0FEF812F902FDF91CF911F91BF
:103D40000F91089582FF14C02E813F818C819D8147
:103D5000281739073CF4E881F981CF01019699834E
:103D6000888310838E819F8101969F838E83E3CF0A
:103D7000E885F985812F0995892BA1F3DACFFA011E
:103D8000AA27283051F1203181F1E8946F936E7F9A
:103D90006E5F7F4F8F4F9F4FAF4FB1E03ED0B4E08B
:103DA0003CD0670F781F891F9A1FA11D680F791FCC
:103DB0008A1F911DA11D6A0F711D811D911DA11DDD
:103DC00020D009F468943F912AE0269F11243019ED
:103DD000305D3193DEF6CF010895462F4770405D88
:103DE0004193B3E00FD0C9F7F6CF462F4F70405D37
:103DF0004A3318F0495D31FD4052419302D0A9F792
:103E0000EACFB4E0A6959795879577956795BA958B
:103E1000C9F700976105710508959B01AC010A2E51
:103E200006945795479537952795BA95C9F7620F28
:103E3000731F841F951FA01D089510E0C2E6D0E0F7
:103E400004C0FE010E94381A2196C336D107C9F773
:043E5000F894FFCF14
:103E540090010000960380003130330047656D699E
:103E64006E69466C617450616E656C50726F0005CA
:103E740002C2010603BC02010001000001010000AE
:103E8400010001010000010000000024018E00BBBC
:103E9400007101EC00CA00DE002A25632573256346
:103EA400002A2563256425630025640025644D25C7
:103EB400644C25644325644425644325644F000011
:00000001FF
